:100000000C947A020C94BE020C94BE020C94BE02B4
:100010000C94BE020C94BE020C94BE020C94BE0260
:100020000C94BE020C94BE020C94620D0C94340E1F
:100030000C94BE020C94BE020C94BE020C94BE0240
:100040000C94BE020C943E220C94BE020C94BE0290
:100050000C94BE020C94D11B0C94BE020C94BE02F4
:100060000C94BE020C94BE020C94BE020C94BE0210
:100070000C94BE020C94BE020C94BE020C94BE0200
:100080000C94BE020C94BE020C94BE020C94BE02F0
:100090000C94BE020C94BE020C94BE020C94BE02E0
:1000A0000C94BE020C94BE020C94BE02A10EC30EB0
:1000B000B10FC30EB10F080F2B0FB10F800F930FAD
:1000C0006212621291129112C712E71218141814D8
:1000D000F2121814A213A2130914181418141214EB
:1000E000AF13AF13AF13AF13AF13AF13AF13AF1300
:1000F000AF13AF13AF13AF13AF13AF13AF13AF13F0
:10010000C113CE13D513DC13E6130000F0A13500A4
:100110002B003171E100015200001E0014000400A8
:100120001D00E0004D001F001A0016001B005000CB
:100130002A0020000800070006004F002C002100C4
:10014000150009001900E2004A00220017000A0009
:10015000050000004C0001542F000000E6000000E4
:100160004900025430000000E6000000290023008E
:100170001C000B00110000006500240018000D0099
:100180001000E2004B0025000C000E00360052006B
:100190002800260012000F0037005100E30027005E
:1001A000130033003800E4004E002E002D0034719F
:1001B000E500025200000100010001000100010001
:1001C00000003A001E0220022202010001003B0052
:1001D0001F0221022302010001003C002F0226021F
:1001E0002F00010001003D00300227023000010015
:1001F00001003E003102350035020000010001001F
:1002000001000000010000000100010001000000E9
:100210000100000001003F005200510024020000D4
:1002200001004000240021001E00270001004100C1
:10023000250022001F0027000100420026002300A5
:10024000200037000100430025022E0231002E005D
:100250000100440045000100010001000000010010
:100260000100010001000100000001000100010087
:1002700001000100010001000100F2000100010085
:1002800001000100F000F1000100F4000100010094
:100290000100F3000100F500010001000100010070
:1002A0000100000001000100010000000100000049
:1002B0000100010001000000010000000100010038
:1002C0000100010001000000010001000100010027
:1002D0000100A9000100010001000100AC00AA001A
:1002E000B600010001000100AB00A8000100010000
:1002F0000100010001000100010001000100AE0049
:1003000001000100000016034500720067006F0045
:1003100044006F007800200045005A0000001603DA
:100320004500720067006F0044006F0078002000F5
:1003300045005A0000000403090409026D0004018D
:1003400000A0FA09040000010301010009211101C4
:100350000001223F000705810308000A090401008B
:100360000103010200092111010001224D000705CE
:10037000820308000A0904020001030000000921A9
:10038000110100012236000705830308000A090451
:1003900003000103000000092111010001223900BE
:1003A000070584031000011201100100000008ED90
:1003B000FE071301000102000105010906A1010564
:1003C0000719E029E7150025019508750181020547
:1003D000081901290595057501910295017503918B
:1003E0000105071900297715002501957875018108
:1003F00002C005010980A101850216010026B7008F
:100400001A01002AB700751095018100C0050C097A
:1004100001A1018503160100269C021A01002A9CF5
:1004200002751095018100C005010902A1010901B1
:10043000A10005091901290515002501950575017A
:10044000810295017503810105010930093115818A
:10045000257F95027508810609381581257F95014C
:1004600075088106050C0A38021581257F950175EE
:10047000088106C0C005010906A101050719E02988
:10048000E715002501950875018102950175088120
:100490000105081901290595057501910295017558
:1004A0000391010507190029FF150025FF95067521
:1004B000088100C0000000000000000000000001F2
:1004C0000204060A0F17202C3A4A5D71879DB3C7B4
:1004D000DAE9F5FCFFFCF5E9DAC7B39D87715D4AFF
:1004E0003A2C20170F0A0604020100000000000049
:1004F0000000000011241FBECFEFDAE0DEBFCDBF49
:1005000004B603FE24C08091FB019091FC01A091F0
:10051000FD01B091FE018730904BA740B04BB9F47C
:100520001092FB011092FC011092FD011092FE014D
:1005300014BE84B7877F84BF88E10FB6F894809398
:100540006000109260000FBEE0E0FFE3099511E04B
:10055000A0E0B1E0EAE0F8E402C005900D92A43317
:10056000B107D9F711E0A4E3B1E001C01D92AB3FA0
:10057000B107E1F70E94A60A0C9403240C94000032
:100580001092B9008AE08093B800089594EA90939D
:10059000BC009091BC0097FFFCCF9091B900987F70
:1005A000983021F0903111F081E008958093BB00E4
:1005B00084E88093BC008091BC0087FFFCCF8091D1
:1005C000B900887F883111F0803471F780E0089598
:1005D00084E98093BC008091BC0084FDFCCF089529
:1005E0008093BB0084E88093BC008091BC0087FFAF
:1005F000FCCF9091B900987F81E0983209F480E0B7
:10060000089584E88093BC008091BC0087FFFCCFF4
:100610008091BB00089580910101811115C080E493
:100620000E94C6028093010181110CC082E10E94E8
:10063000F00280930101811105C08FEF0E94F0024A
:10064000809301010E94E80284B1807F84B985B162
:10065000807F85B98AB1837F8AB98BB1837F8BB95B
:100660003E98469808950E94C604809301010E9416
:100670000B0380B38C7080BB81B3836F81BBA5E318
:10068000B1E0E3E4F1E08EE08E0F11921D928E1343
:10069000FCCF0C94B004BF92CF92DF92EF92FF9206
:1006A0000F931F93CF93DF9380910101882379F0FB
:1006B000809134018F5F80933401811108C00E94C2
:1006C000C60480930101811102C00E94580405E311
:1006D00011E0C0E0D0E0DD24D39482E0C82EEE2407
:1006E000E394F12CC730D10500F58091010181110F
:1006F00064C080E40E94C60280930101811112C08F
:1007000082E10E94F0028093010181110BC0C701B8
:100710000C2E01C0880F0A94EAF780950E94F0021F
:10072000809301010E94E80248C0CA30A1F028F479
:10073000C83059F0C93061F005C0CC3089F070F094
:10074000CD3089F0209A289810C0219A29980DC0A0
:10075000229A2A980AC0239A2B9807C0529A01C05D
:10076000539A5B9802C03E9A469890EA9A95F1F7A0
:100770009FB1799902C082E001C080E091709D250F
:10078000982B7C9902C084E001C080E0892B7D9980
:1007900002C038E001C030E0832B7E9902C020E126
:1007A00001C020E0822B9FB19095991F9927991F36
:1007B0009295990F907E892B0FC080910101811134
:1007C00049C080E40E94C60280930101882379F128
:1007D000B12C0E94E8028B2DF8019081981719F036
:1007E0008083C09200010E940B0321960F5F1F4F70
:1007F000CE30D10509F076CF80910001882361F1D8
:10080000815080930001882339F08FE99FE00197A0
:10081000F1F700C0000020C0A3E4B1E0E5E3F1E09F
:10082000CF01825F91919D938E13FCCF15C083E120
:100830000E94F002809301018111CACF81E40E94DD
:10084000C602809301018111C3CF0E940103B82E1B
:10085000B094BFCF80E0C0CF0E94560481E0DF910A
:10086000CF911F910F91FF90EF90DF90CF90BF90AD
:100870000895E82FF0E0ED5BFE4F80810895089524
:100880000F931F93CF93DF93C3E4D1E010E00C2FBD
:10089000025F899190E00E94F71A180F0C13F9CFAC
:1008A000812FDF91CF911F910F9108950C94260510
:1008B00056985E9825982D9826982E9827982F98C8
:1008C0008FEF90E0909389008093880090938B0045
:1008D00080938A0090938D0080938C00259A2D9AA6
:1008E0002FEF80E792E0215080409040E1F700C078
:1008F0000000269A2E9A2FEF80E792E02150804048
:100900009040E1F700C00000279A2F9A2FEF80E770
:1009100092E0215080409040E1F700C0000025980F
:100920002D982FEF80E792E0215080409040E1F732
:1009300000C0000026982E982FEF80E792E021500B
:1009400080409040E1F700C0000027982F9856980B
:100950005E9825982D9826982E9827982F98089578
:1009600089EA8093800089E08093810024982C9804
:100970003F988AB18F748AB96E98479A8BB1806B11
:100980008BB9769A0E9458040C94250580E28093D6
:1009900001018091510181110EC00E94C00281E0CD
:1009A000809351012FEF83ED90E3215080409040E0
:1009B000E1F700C0000080E40E94C60280930101BC
:1009C00081112EC00E94F00280930101811128C084
:1009D0000E94F00280930101811122C08FE30E94E6
:1009E000F0028093010181111BC00E94E80280E4A3
:1009F0000E94C60280930101811112C08CE00E9406
:100A0000F0028093010181110BC00E94F0028093DB
:100A10000101811105C08FE30E94F0028093010162
:100A20000E94E80280910101089561110BC0FC0150
:100A30008281882321F085EE0E94061103C085EE95
:100A40000E94CE1180E090E0089508956091BD016C
:100A50007091BE018091BF019091C0010E94031B63
:100A600056985E9825982D9826982E9827982F9816
:100A7000813019F0823021F00895259A2D9A089539
:100A8000269A2E9A089581E0089581E008950C94A5
:100A9000450508950F931F93CF93DF938C01FC01BD
:100AA000C081D181CE010E947C19BE010E94F30554
:100AB000EC01B8010E944705882309F48DC0F801B4
:100AC0008281882309F44AC080915D0181111FC091
:100AD000C431F0E5DF0709F051C00E94490581E00B
:100AE00080935D010E949B1B90935C0180935B014E
:100AF0001092540110925601109255011092580113
:100B00001092570110925A011092590165C08091BC
:100B10005B0190915C010E94A71B883C910570F4D9
:100B200080915401E82FF0E0EE0FFF1FEB5AFE4FCB
:100B3000D183C0838F5F809354014EC0C43880E559
:100B4000D80721F0C538D04501F13AC0F8018281BB
:100B5000882341F01092520182E01EC0C438E0E5C3
:100B6000DE0759F580915201811106C086E20E948C
:100B7000061186E20E94CE1182E01CC0C438F0E566
:100B8000DF0741F3C538D045D9F4F80182818823C5
:100B900031F01092530180E20E941D121DC080911D
:100BA0005301811106C087E20E94061187E20E946C
:100BB000CE1180E20E9424120FC0C538D04529F31F
:100BC00081E08093520180935301C801DF91CF915E
:100BD0001F910F910C94430580E0DF91CF911F91FD
:100BE0000F910895089596E0799FF001112494E5FE
:100BF000899FE00DF11D1124E60FF11DEE0FFF1F7F
:100C0000E25FFE4F859194910895880F991FFC0132
:100C1000E657F040859194910895880F991FFC0143
:100C2000E65FFE4F8591949108950F931F93CF93A4
:100C3000DF93EC01811520E3920750F5C11580E2A6
:100C4000D80708F0C3C0CB3BD10590F4C83AD10512
:100C500008F06AC0C53AD10508F05BC0C430D105C0
:100C600008F0D0C1219709F0CAC101E010E00AC222
:100C7000CF3FD10511F008F0C5C1C03FD10508F044
:100C8000A2C0CE01805E9109089708F4BBC1B7C12C
:100C9000C13090E5D90709F4A2C020F5C0318FE436
:100CA000D80770F4C11590E4D90708F094C0C115B5
:100CB00021E3D20708F0A3C1DD278E01106CE2C149
:100CC000C115D04509F09BC10E9483148FEF94E3B6
:100CD0002CE0815090402040E1F700C000000E94CD
:100CE000F61BD0C1C11597E5D90758F4C03121E5ED
:100CF000D20708F01CC1C43180E5D80708F475C0DC
:100D00007EC1CE0190578115904108F078C1DF7007
:100D100073C1C53AD10509F477C1C63AD10509F0C6
:100D200076C102E810E4AEC1C83AD10509F472C137
:100D3000C93AD10509F471C1CA3AD10509F470C1A3
:100D4000CB3AD10509F46FC1CC3AD10509F46EC193
:100D5000CD3AD10509F46DC1C03BD10509F46CC190
:100D6000CE3AD10509F46BC1CF3AD10509F46AC175
:100D7000C13BD10509F469C1C23BD10509F468C181
:100D8000C33BD10509F467C1C43BD10509F466C171
:100D9000C53BD10509F465C1C63BD10509F464C161
:100DA000C73BD10509F463C1C83BD10509F462C151
:100DB000C93BD10509F461C1CA3BD10509F460C141
:100DC00000E014E45FC18E0110655CC1CE019F702C
:100DD0000E940D0658C1DF708E01106A53C18091C8
:100DE000DA0181608093DA014DC10E949B1D81115F
:100DF00002C00E94811D0E94B81D90E09093FB01EB
:100E00008093FA01C23080E5D80721F48091FA017D
:100E1000816086C0C43090E5D90721F48091FA0141
:100E200082607EC0C63020E5D20721F48091FA01AD
:100E3000846076C0C83080E5D80719F48091FA0143
:100E400027C0CA3090E5D90721F48091FA0180616A
:100E500067C0CC3020E5D20721F48091FA0180628E
:100E60005FC0CE3080E5D80721F48091FA0180641C
:100E700057C0C03190E5D90721F48091FA0180680C
:100E80004FC0C23120E5D20729F48091FA01846075
:100E9000886046C0C33080E5D80721F48091FA010C
:100EA0008E7F3EC0C53090E5D90721F48091FA01CC
:100EB0008D7F36C0C73020E5D20721F48091FA013A
:100EC0008B7F2EC0C93080E5D80719F48091FA01D4
:100ED00026C0CB3090E5D90721F48091FA018F7EAE
:100EE0001FC0CD3020E5D20721F48091FA018F7D1B
:100EF00017C0CF3080E5D80721F48091FA018F7BAD
:100F00000FC0C13190E5D90721F48091FA018F77A4
:100F100007C0C331D04531F48091FA018B7F877FC0
:100F20008093FA018091FA010E94BC1DABC08D2F05
:100F300099278F70992781309105D9F49E012370EC
:100F4000332702C0880F991F2A95E2F79C688E010B
:100F500044E0000F111F4A95E1F700271370802B22
:100F6000912B53E0CC0FDD1F5A95E1F7C076DD27BA
:100F70002FC08230910531F4DC2FCC278E01016F18
:100F8000106A80C08330910569F4CE01837099277F
:100F900001E010E002C0000F111F8A95E2F7C801BE
:100FA0009C680FC084309105B9F4CE0183709927F5
:100FB00001E010E002C0000F111F8A95E2F7C8019E
:100FC0009A6823E0CC0FDD1F2A95E1F7C07ED77029
:100FD0008C010C2B1D2B56C08530910531F4DC2F74
:100FE000CC278E01046F106A4DC0069709F04AC0E5
:100FF000CF71DD27DC2FCC278E01106243C000E0CB
:1010000010E040C08E013EC001E810E43BC003E8A0
:1010100010E438C002EE14E435C009EE14E432C026
:101020000AEE14E42FC005EB14E42CC006EB14E424
:1010300029C007EB14E426C00CEC14E423C00DEC2B
:1010400014E420C003E815E41DC00AE815E41AC042
:1010500002E915E417C004E915E414C001E216E43E
:1010600011C003E216E40EC004E216E40BC005E270
:1010700016E408C006E216E405C007E216E402C062
:101080000AE216E4C801DF91CF911F910F910895F4
:1010900096E0799FF001112494E5899FE00DF11D00
:1010A0001124E60FF11DEE0FFF1FE25FFE4F859149
:1010B0009491803E9105E0F4803C910558F5813390
:1010C000910509F46FC048F48932910509F463C0B1
:1010D0008A32910509F46DC072C089339105E9F037
:1010E00082389105D1F08533910509F44DC067C070
:1010F000833E910581F138F4803E9105B9F0823E3E
:101100009105D9F05CC0863E910561F1873E91055D
:10111000A1F155C00E94050608952091FA0120FD15
:1011200002C021FF4CC080EE90E049C08091FA01DE
:1011300080FFF9CF89E390E042C08091FA0182FFFD
:101140000EC08091FA0184FF03C080E090E037C0B8
:1011500083EE90E034C08091FA0182FFF2CF82EEFC
:1011600090E02DC08091FA0183FF0BC08091FA01BD
:1011700084FDEBCF87EE90E022C08091FA0183FFDF
:10118000F5CF86EE90E01BC08091FA0185FF07C085
:1011900089E290E014C08091FA0185FFF9CF85E3E0
:1011A00090E00DC08091FA0186FF07C08AE290E0CE
:1011B00006C08091FA0186FFF9CF81E390E00E949A
:1011C0001506089508950C94E20880916E01089523
:1011D000CF93DF9300D01F92CDB7DEB79C018091F3
:1011E000F101843019F593E099833B832A8390932E
:1011F000E9008FEF9091E800815095FD06C095EDD4
:101200009A95F1F700008111F5CF8091E80085FFF4
:101210000DC040E050E063E070E0CE0101960E9416
:10122000520B8091E8008E778093E8000F900F902A
:101230000F90DF91CF910895CF93DF9300D01F924D
:10124000CDB7DEB72091F101243021F522E02983CA
:101250009B838A8383E08093E9008FEF9091E8007D
:10126000815095FD06C095ED9A95F1F7000081112A
:10127000F5CF8091E80085FF0DC040E050E063E0CD
:1012800070E0CE0101960E94520B8091E8008E77AB
:101290008093E8000F900F900F90DF91CF91089509
:1012A0002091F1012430F1F422E02093E9002FEFA6
:1012B0003091E800215035FD06C035ED3A95F1F743
:1012C00000002111F5CF2091E80025FF0BC040E080
:1012D00050E065E070E00E94520B8091E8008E774C
:1012E0008093E8000895CF93DF93EC019091F10192
:1012F000943009F046C080910C018823D9F0809188
:101300000D018823B9F09093E9008FEF9091E800E8
:10131000815095FD06C095E19A95F1F70000811185
:10132000F5CF8091E80085FF2CC040E050E060E1FF
:1013300070E017C081E08093E9008FEF9091E800A2
:10134000815095FD06C095ED9A95F1F70000811149
:10135000F5CF8091E80085FF14C040E050E068E0E0
:1013600070E0CE010E94520B8091E8008E7780934E
:10137000E80080E1FE01AEE5B1E001900D928A95B2
:10138000E1F7DF91CF9108958091F001811109C0BB
:101390000E94E70C0E94440D8091E20084608093DB
:1013A000E20008951092F001089508950C942B2204
:1013B0000E948C1B0E9431220E94EA0F0C94E308C9
:1013C00042E061EC81E00E94610C42E061EC82E06D
:1013D0000E94610C42E061EC83E00E94610C42E1FA
:1013E00061EC84E00C94610C8091F301833009F48A
:1013F00055C030F4813071F0823009F48EC0089508
:101400008A3009F47AC08B3009F460C0893009F061
:101410009CC020C08091F201813A09F096C0809171
:10142000E800877F8093E8008091F6019091F701B2
:10143000892B21F460E18EE591E003C060E080E05B
:1014400090E070E00E949D0B8091E8008B77809384
:10145000E80008958091F201813209F076C0809110
:10146000F6019091F701009719F0039709F06DC00C
:101470008091E800877F8093E8008091E80082FDFA
:1014800005C08091F1018111F8CF5FC08091F1001A
:1014900080936E018091E8008B7753C08091F201B8
:1014A000813A09F052C08091F6019091F701892BA1
:1014B00009F04BC08091E800877F8093E80080911D
:1014C000E80080FFFCCF80910C0136C08091F201D2
:1014D0008132D9F58091F6019091F701892BA9F518
:1014E0008091E800877F8093E8000E94960C8091AD
:1014F000F40180930C010C9483148091F2018132E9
:1015000021F58091E800877F8093E8000E94960C87
:101510008091F50180936F0108958091F201813AE5
:10152000A1F48091E800877F8093E8008091E80033
:1015300080FFFCCF80916F018093F1008091E800E3
:101540008E778093E8000C94960C089584B7877F7B
:1015500084BF88E10FB6F894809360001092600019
:101560000FBE90E080E80FB6F894809361009093EE
:1015700061000FBE0E9439100E94E70C0E94440DCA
:101580008091E20084608093E20078940E94CA0F08
:101590000E943B1082E091E00E94E50F0E94192218
:1015A0008091F101853069F40E94531B8091EF0115
:1015B0008823B1F30E947E1B882391F30E943C0B89
:1015C000EFCF0E944110ECCF292F33272330310574
:1015D000C9F064F42130310581F02230310509F081
:1015E00043C08DE690E02AE333E042C0213231056A
:1015F000F1F02232310541F137C082E190E027EA73
:1016000033E036C099278130910541F08230910551
:1016100041F0892B49F5E6E3F3E005C0EEE1F3E0A4
:1016200002C0E6E0F3E0849190E09F0121C06430C5
:10163000D8F4E62FF0E0EE0FFF1FEE5DFE4F2081A5
:10164000318189E090E014C0643070F470E0FB01F7
:10165000EE0FFF1FE65EFE4F20813181FB01EA5E47
:10166000FE4F808190E004C080E090E020E030E018
:10167000FA0131832083089580E189BD82E189BD2B
:1016800009B400FEFDCF8091D8008F7D8093D800F3
:101690008091E00082608093E0008091E00081FD15
:1016A000FCCF0895CF92DF92EF92FF920F931F939A
:1016B000CF93DF93EC018B016A010E94B50C81117D
:1016C00033C0C114D10439F0F60180819181081B27
:1016D000190BC80FD91FE12CF12C0115110519F1B7
:1016E0008091E80085FD16C08091E8008E77809398
:1016F000E800C114D10449F0F60180819181E80E1F
:10170000F91EF182E08285E00FC00E94B50C8823AB
:1017100021F30AC089918093F10001501109FFEF74
:10172000EF1AFF0ADACF80E0DF91CF911F910F917E
:10173000FF90EF90DF90CF9008952091F8013091C5
:10174000F9012617370748F06115710539F4209122
:10175000E8002E772093E80001C0B90140E0611550
:101760007105A9F12091F101222309F443C025302C
:1017700009F442C02091E80023FD40C02091E80018
:1017800022FD32C02091E80020FFE9CF4091F30014
:101790002091F20030E0342BFC01CF01611571057E
:1017A00059F02830310540F481918093F100615067
:1017B00071092F5F3F4FF1CF41E02830310509F02B
:1017C00040E02091E8002E772093E800C8CF411137
:1017D000C9CF0AC08091F101882361F0853061F0A2
:1017E0008091E80083FD0AC08091E80082FFF2CF7B
:1017F00080E0089582E0089583E0089581E00895EF
:101800002091F8013091F9012617370748F061154A
:10181000710539F42091E8002E772093E80001C08B
:10182000B901FC0120E06115710591F18091F10190
:10183000882309F440C0853009F43FC08091E80056
:1018400083FD3DC08091E80082FD2FC08091E800BB
:1018500080FFE9CF2091F3008091F20090E0922B7D
:101860006115710559F08830910540F42491209359
:10187000F1003196615071090196F2CF21E008978D
:1018800009F020E08091E8008E778093E800CBCFCC
:101890002111CCCF0AC08091F101882361F08530FD
:1018A00061F08091E80083FD0AC08091E80082FF2A
:1018B000F2CF80E0089582E0089583E0089581E00A
:1018C0000895982F973058F59093E900981739F0BC
:1018D0007091EC002091ED005091F00003C0242F96
:1018E000762F50E021FF19C03091EB003E7F3093FE
:1018F000EB003091ED003D7F3093ED003091EB0037
:1019000031603093EB007093EC002093ED00509326
:10191000F0002091EE0027FF07C09F5FD3CF8F70AC
:101920008093E90081E0089580E008958091F201BC
:1019300087FF11C08091E80082FD05C08091F10110
:101940008111F8CF11C08091E8008B770BC0809196
:10195000F101882349F08091E80080FFF8CF809161
:10196000E8008E778093E80008952091E40030919C
:10197000E50095E64091EC00842F817040FF22C085
:101980008091E80080FD1CC08091F101882391F0D6
:10199000853091F08091EB0085FD10C04091E4000E
:1019A0005091E5004217530729F39A01915011F71E
:1019B00084E0089582E0089583E0089581E0089529
:1019C00080E008954091E80042FFDECF08950E9434
:1019D000550D0E945D0DE0EEF0E080818160808316
:1019E000E8EDF0E080818F77808319BCA7EDB0E04F
:1019F0008C918E7F8C9380818F7E80831092F001FA
:101A000008950F931F93CF93DF930E94550D0E946B
:101A10005D0DC8EDD0E088818F77888388818068EC
:101A2000888388818F7D888319BC1092F101109280
:101A3000ED011092EF011092EE0100EE10E0F801BE
:101A400080818B7F808388818160888342E060E031
:101A500080E00E94610CE1EEF0E080818E7F808367
:101A6000E2EEF0E080818160808380818860808305
:101A7000F80180818E7F8083888180618883DF91F7
:101A8000CF911F910F910895E8EDF0E080818F7E56
:101A90008083E7EDF0E080818160808384E082BF15
:101AA00081E08093F0010C94010DE8EDF0E080817D
:101AB0008E7F80831092E20008951092DA001092D7
:101AC000E10008951F920F920FB60F9211242F93E9
:101AD0003F934F935F936F937F938F939F93AF93B6
:101AE000BF93EF93FF938091E10082FF0BC0809141
:101AF000E20082FF07C08091E1008B7F8093E100CC
:101B00000E94C90F8091DA0080FF1FC08091D80029
:101B100080FF1BC08091DA008E7F8093DA00809175
:101B2000D90080FF0DC080E189BD82E189BD09B483
:101B300000FEFDCF81E08093F1010E94C40905C041
:101B400019BC1092F1010E94D2098091E10080FF3E
:101B500019C08091E20080FF15C08091E2008E7F65
:101B60008093E2008091E20080618093E2008091A6
:101B7000D80080628093D80019BC85E08093F10181
:101B80000E94D6098091E10084FF30C08091E2007C
:101B900084FF2CC080E189BD82E189BD09B400FECB
:101BA000FDCF8091D8008F7D8093D8008091E10097
:101BB0008F7E8093E1008091E2008F7E8093E2002F
:101BC0008091E20081608093E2008091ED018823A2
:101BD00011F084E007C08091E30087FD02C081E03E
:101BE00001C083E08093F1010E94D8098091E10057
:101BF00083FF29C08091E20083FF25C08091E1002E
:101C0000877F8093E10082E08093F1011092ED01E3
:101C10008091E1008E7F8093E1008091E2008E7FD1
:101C20008093E2008091E20080618093E20042E0D4
:101C300060E080E00E94610C8091F00088608093F9
:101C4000F0000E94D509FF91EF91BF91AF919F9154
:101C50008F917F916F915F914F913F912F910F9055
:101C60000FBE0F901F9018951F920F920FB60F92F4
:101C700011242F933F934F935F936F937F938F9391
:101C80009F93AF93BF93CF93DF93EF93FF93C09155
:101C9000E900CF708091EC00D82FD17080FDD0E8A2
:101CA0001092E9008091F000877F8093F000789493
:101CB0000E94780E1092E9008091F0008860809375
:101CC000F000CD2BCF70C093E900FF91EF91DF9131
:101CD000CF91BF91AF919F918F917F916F915F91C4
:101CE0004F913F912F910F900FBE0F901F9018951D
:101CF0001F93CF93DF93CDB7DEB7AA970FB6F894B3
:101D0000DEBF0FBECDBFE2EFF1E088E08E0F909115
:101D1000F10091938E13FBCF0E94F4098091E800AB
:101D200083FF1FC18091F2019091F301492F50E090
:101D30004A30510508F015C1FA01EA5AFF4F0C94D8
:101D4000B323803881F0823809F00BC18091F6010D
:101D50008F708093E9008091EB0085FB882780F9E4
:101D60001092E90006C08091EE019091EF0191116F
:101D700082609091E800977F9093E8008093F10053
:101D80001092F100C8C0282F2D7F09F0EAC08823E7
:101D900019F0823061F0E5C08091F401813009F0E2
:101DA000E0C0933009F080E08093EF012BC0809178
:101DB000F401811127C08091F6018F7009F4D1C020
:101DC0008093E9002091EB0020FF1CC0933021F4A8
:101DD0008091EB00806214C09091EB009061909331
:101DE000EB0021E030E0A90102C0440F551F8A95A5
:101DF000E2F74093EA001092EA008091EB008860DD
:101E00008093EB001092E9008091E800877F86C004
:101E10008111A7C01091F4011F778091E3008078B1
:101E2000812B8093E3008091E800877F8093E80016
:101E30000E94960C8091E80080FFFCCF8091E30027
:101E400080688093E300111102C082E001C083E04A
:101E50008093F10186C08058823008F082C0809162
:101E6000F4019091F5018C3D53E0950779F583E0FD
:101E70008A838AE289834FB7F894DE01139620E0C3
:101E80003EE051E2E32FF0E050935700E49120FF51
:101E900003C0E295EF703F5FEF708E2F90E0EA3065
:101EA00010F0C79601C0C0968D939D932F5F24318B
:101EB00049F74FBF8091E800877F8093E8006AE28E
:101EC00070E0CE0101960E949D0B14C0AE014F5FE1
:101ED0005F4F6091F6010E94E40ABC01009709F48B
